:1000000008308A0066280000FF00030E8301A1006B
:100010000A08A0008A010408A2007708A300780853
:10002000A4007908A5007A08A6007B08A70083131E
:1000300083128B1E1D280B1936288C308400801EDD
:1000400023288C1A3928220884002308F700240862
:10005000F8002508F9002608FA002708FB00200808
:100060008A00210E8300FF0E7F0E09008A110A12FA
:100070005C288A110A1271280A108A100A11820754
:100080005334443452342D343134343400340A106F
:100090008A100A118207493464346C3465340034A0
:1000A0000A108A100A118207523475346E346E3485
:1000B00069346E3467340034AA0803196528AB0B21
:1000C0006428AA010E30AB0067280E30AB00A908E7
:1000D00003196D28A90B6D2828140B118A110A1217
:1000E0002328981C7528181218162C08AC0A023EF2
:1000F0008316A40083121A08F80010308316240710
:10010000840078088317800083131F308312AC05A6
:100110008C128A110A122328003083168800831259
:100120002E0888008714051A9728281C9328FF306A
:1001300083168800831287100034A8112810D3304A
:1001400087004630A900051EA728281CA328D03008
:1001500087002818AE28FC30AE058C200034051E20
:10016000B328281CAF282818F028F83005050738D0
:100170008500831621088312860085118515F830C5
:100180000505063885008316200883128600851130
:100190008515F8300505043885007408860085113A
:1001A0008515F8300505033885007308860085112C
:1001B0008515F8300505023885007208860085111E
:1001C0008515F83005050138850071088600851110
:1001D0008515F830050585007008860085118515A0
:1001E0000034051EF528281CF1282818FE28AE1416
:0E01F0008C20AE10051EFE28281CFA280034B4
:02020E00F301FA
:10021000F201F101F0014F08BF004E08BE004D0889
:10022000BD004C08BC004B08C3004A08C200490886
:10023000C1004808C0000322440DBC00450DBD00AC
:10024000460DBE00470DBF00BC0DBD0DBE0DBF0D60
:10025000BC0DBD0DBE0DBF0DBC0DBD0DBE0DBF0D4A
:10026000F030BC0503223C0EF300F030F305440DE2
:10027000BC00450DBD00460DBE00470DBF00BC0DC6
:10028000BD0DBE0DBF0DBC0DBD0DBE0DBF0DBC0D1A
:10029000BD0DBE0DBF0DF030BC0503223C08F307B9
:1002A000440DBC00450DBD00460DBE00470DBF000E
:1002B000BC0DBD0DBE0DBF0DBC0DBD0DBE0DBF0DEA
:1002C000BC0DBD0DBE0DBF0DF030BC0503223C0EB4
:1002D000F200F030F205440DBC00450DBD00460DA6
:1002E000BE00470DBF00BC0DBD0DBE0DBF0DBC0D4A
:1002F000BD0DBE0DBF0DBC0DBD0DBE0DBF0DF03053
:10030000BC0503223C08F207440DBC00450DBD00AE
:10031000460DBE00470DBF00BC0DBD0DBE0DBF0D8F
:10032000BC0DBD0DBE0DBF0DBC0DBD0DBE0DBF0D79
:10033000F030BC0503223C0EF100F030F105440D15
:10034000BC00450DBD00460DBE00470DBF00BC0DF5
:10035000BD0DBE0DBF0DBC0DBD0DBE0DBF0DBC0D49
:10036000BD0DBE0DBF0DF030BC0503223C08F107EA
:10037000440DBC00450DBD00460DBE00470DBF003D
:10038000BC0DBD0DBE0DBF0DBC0DBD0DBE0DBF0D19
:10039000BC0DBD0DBE0DBF0DF030BC0503223C0EE3
:1003A000F000F030F005440DBC00450DBD00460DD9
:1003B000BE00470DBF00BC0DBD0DBE0DBF0DBC0D79
:1003C000BD0DBE0DBF0DBC0DBD0DBE0DBF0DF03082
:1003D000BC0503223C08F00703308316A100A000EF
:1003E0008312AF200034051EF729281CF329281892
:0A03F000FC292E148C202E1000347E
:0A040600C701C601C501C40140088A
:10041000C4024108031C410FC5024208031C420FDD
:10042000C6024308031C430FC702BF0D0730B300C9
:100430003F0DC40DC50DC60DC70D40083F1C2E2A2B
:10044000C4024108031C410FC5024208031C420FAD
:10045000C6024308031C430FC7023B2AC4074108D6
:100460000318410FC50742080318420FC607430887
:100470000318430FC707BF0DB30B182A3E0DC40D59
:10048000C50DC60DC70D40083F1C542AC4024108C3
:10049000031C410FC5024208031C420FC602430859
:1004A000031C430FC702612AC40741080318410F08
:1004B000C50742080318420FC60743080318430F35
:1004C000C707BE0D0730B3003E0DC40DC50DC60DE8
:1004D000C70D40083E1C7A2AC4024108031C410F84
:1004E000C5024208031C420FC6024308031C430F07
:1004F000C702872AC40741080318410FC5074208ED
:100500000318420FC60743080318430FC707BE0D61
:10051000B30B642A3D0DC40DC50DC60DC70D4008B3
:100520003E1CA02AC4024108031C410FC502420818
:10053000031C420FC6024308031C430FC702AD2A27
:10054000C40741080318410FC50742080318420FAA
:10055000C60743080318430FC707BD0D0730B30094
:100560003D0DC40DC50DC60DC70D40083D1CC62A66
:10057000C4024108031C410FC5024208031C420F7C
:10058000C6024308031C430FC702D32AC40741080D
:100590000318410FC50742080318420FC607430856
:1005A0000318430FC707BD0DB30BB02A3C0DC40D94
:1005B000C50DC60DC70D40083D1CEC2AC4024108FC
:1005C000031C410FC5024208031C420FC602430828
:1005D000031C430FC702F92AC40741080318410F3F
:1005E000C50742080318420FC60743080318430F04
:1005F000C707BC0D0730B3003C0DC40DC50DC60DBB
:10060000C70D40083C1C122BC4024108031C410FBB
:10061000C5024208031C420FC6024308031C430FD5
:10062000C7021F2BC40741080318410FC507420822
:100630000318420FC60743080318430FC707BC0D32
:10064000B30BFC2A3C18322B4008C407410803189E
:10065000410FC50742080318420FC6074308031895
:10066000430FC7070034051E372B281C332B2818CF
:10067000722BAC080319722B83168C120230831272
:10068000AC072C0803179000C03091000313B4018D
:1006900000308316880083122C0834020318682B5C
:1006A0003408B40AFC0010307C078400831700086B
:1006B0008313FD0088000714051A602B281C5C2B8F
:1006C0000710051E652B281C612B83164B2B8312EC
:1006D000FF30831688008312AC0183168C168312B8
:1006E000091009148A150A12432A39083802031915
:1006F000A82B8316981CA92B8312281F812B871DDA
:10070000A82B3908B90AFC0090307C0784008317B5
:1007100000088313B4001F30B905B7080319A62BCE
:100720008316181083123408B500B500350C350651
:10073000B500B50CB50CB506350EB506350BA12BBD
:10074000B509351CA62B831618148312340899009A
:10075000831683128A150A12462AA03084000008E4
:100760000319BF2B0130F800F701F70BB52BF80B7D
:10077000B42B3230F700F70BBB2B800BB22B0034BD
:10078000A810AF014630A900D108031D392ED101B0
:100790005208F7005308FA007A08031DD32B1830CB
:1007A00077020319262C7A08031DDA2B20307702F2
:1007B00003198D2C7A08031DE12BB0307702031941
:1007C0009A2C7A08031DE82B3830770203192A2D5A
:1007D0007A08031DEF2B4030770203194B2D0330AD
:1007E0007A02031DF62BF70803197B2D02307A02DB
:1007F000031DFD2BF7080319BF2D02307A02031DDC
:10080000052C013077020319FE2D02307A02031DF8
:100810000D2C0230770203190B2E02307A02031DD1
:10082000152C0330770203192C2E02307A02031D97
:100830001D2C043077020319312E02307A02031D79
:10084000252C053077020319322E332E0830D000C4
:100850005508023C031D8B2CAD0154087F39003A2A
:10086000031D342C8516352C85126030AE04D41F40
:100870003B2C2E13442CAE120130F00003308316B3
:10088000A100A0018312AF205708B100B108031DD9
:100890004B2C0130B1003108803C0318512C8030C2
:1008A000B100A8127730AE055608003A0319652C3E
:1008B000013A0319692C033A03196D2C013A031903
:1008C000722C073A0319772C7D2CB101B001AE15BB
:1008D000822C01303107B000822CA816013031077C
:1008E000B000822C01303107B000AE17822CA81660
:1008F00001303107B000AE17822CA8160130310745
:10090000B000822C8C20F12019308316A0008312B5
:10091000AD23A8158C2CA811372E0A30D000D40195
:100920005808CF005708CE005608CD005508CC0017
:100930000721372E0930D000D40155084802031D85
:10094000AD2C56084902031DAD2C57084A02031D61
:10095000AD2C58084B020319292D5808CB00570815
:10096000CA005608C9005508C800103003178D008A
:100970000313480803178C0083168C130C1583127D
:1009800003130B08F7008B138316031755308D00E4
:10099000AA308D008C148C18CB2C0C117708831284
:1009A00003138B04113003178D0003134908031739
:1009B0008C0083168C130C15831203130B08F7009D
:1009C0008B138316031755308D00AA308D008C14BD
:1009D0008C18E82C0C117708831203138B04123047
:1009E00003178D0003134A0803178C0083168C131A
:1009F0000C15831203130B08F7008B1383160317D0
:100A000055308D00AA308D008C148C18052D0C11DA
:100A10007708831203138B04133003178D0003131D
:100A20004B0803178C0083168C130C1583120313C9
:100A30000B08F7008B138316031755308D00AA306F
:100A40008D008C148C18222D0C117708831203133F
:100A50008B04372E0630D000D4015508B600360876
:100A6000803A663C031C372DEB30AE05492D360825
:100A7000803A703C031C3F2D2E112E16492D36084E
:100A8000803A7A3C031C472D2E152E12492D143026
:100A9000AE048C20372E0630D000D4015508B600A5
:100AA0003608003A0319612D063A0319642D0A3AF3
:100AB0000319672D1E3A03196A2D0A3A03196D2D81
:100AC0006F2D0430F0006F2D0330F0006F2D0230D9
:100AD000F0006F2D0130F0006F2DF0016F2DF1014E
:100AE000F201F301F40103308316A1000930A000E4
:100AF0008312AF20372E56085A3C031DBB2D570FCB
:100B0000BB2D5808A53C031DBB2DD908031DBB2DCB
:100B1000D508031DBA2D0711051A8C2D0030831638
:100B20008800831250082F020318AC2D2F08AF0A3B
:100B3000503E840000088316A10083128800071429
:100B4000051AA42D281CA02D0710051EA92D281C50
:100B5000A52D8316912D8312FF30831688008312F2
:100B60000B138B138B1BB12D5A30FE00A530FF00E9
:100B70008A010028BE2DD1010230D000372E57083F
:100B8000B700D9080319CA2D2817D8308316870053
:100B9000CC2D83122813831683125B084B3A03195A
:100BA000DB2D6E3A0319DE2D373A0319E12D1B3A7E
:100BB0000319E42DE72D0B30B400EA2D1730B400F3
:100BC000EA2D2F30B400EA2D5F30B400EA2DC0309A
:100BD000B400EA2D34088316990067309800831218
:100BE000B7080319F62DD0309800F82D90309800F2
:100BF000B801B90183168C168312372E83168C1216
:100C000083129801473083169800D03087008312F2
:100C1000B801B901372EC03083168700831207163A
:100C2000571C152E8715A813172E8711A8175808BB
:100C3000BB00BB033B080739F8000130BA00F808D5
:100C40000319262E0310BA0DF80B222EBB0CBB0C79
:100C5000BB0C1F30BB05372ED030831687008312A4
:100C6000372E372E372ED1010230D000372E2815DF
:100C7000E32F5108203C031D5D2FD1015208F700DE
:100C80005308FA007A08031D492E01307702031930
:100C9000892E7A08031D502E0230770203199E2EEA
:100CA0007A08031D572E033077020319C62E7A08DF
:100CB000031D5E2E043077020319CC2E7A08031D23
:100CC000652E053077020319F22E7A08031D6C2E6B
:100CD000063077020319F72E7A08031D732E183099
:100CE000770203192C2F7A08031D7A2E2030770201
:100CF0000319372F7A08031D812EB03077020319AC
:100D0000452F7A08031D882E383077020319512F9A
:100D1000572FFC0104307C07503E84007C083C20A7
:100D2000F80080007C08FC0A043E503E84008008E5
:100D3000031D8A2E04307C07D0005B2FFC017C0849
:100D400003178D0083168C130C1483120C080313E5
:100D5000B4007C08FC0A043E503E84003408800045
:100D600034082F3C0318BC2E34085A3C031CBC2EFC
:100D70007C080A3C03189F2E7C08FC0A043E503E67
:100D80008400800104307C07D0005B2F0630D00047
:100D90000230D400D5015B2F0730D000540BD52E84
:100DA0006430D5000030D600F12EFA3003178D00E4
:100DB0001F308F0083168C170C1400000000831264
:100DC0000C080313D500FB3003178D001F308F0074
:100DD00083168C170C140000000083120C080313F8
:100DE000D6005B2F0530D0003208D4005B2FFC0109
:100DF00054080B3A0319002F073A0319132F272F12
:100E000004307C07503E84007C084720F8008000B6
:100E10007C08FC0A043E503E84008008031D002F1D
:100E200004307C07D00004307C07503E84007C08EE
:100E30005020F80080007C08FC0A043E503E8400EC
:100E40008008031D132F04307C07D0002B2FD10105
:100E50000230D0002B2F5B2F0830D000D401A81D0A
:100E6000342F0230D500362F0130D5005B2F0A30E9
:100E7000D000D4014F08D8004E08D7004D08D60046
:100E80004C08D5000130D9005B2F0930D000D401C7
:100E90004B08D8004A08D7004908D6004808D500B2
:100EA0005B2F0630D000D4013608D5005B2FD1016E
:100EB0000230D0005B2F2815E32F5108403C031D62
:100EC000682F4030D100D1010230D0002815E32F27
:100ED0005108A03C031D872F5408F0005508F1006D
:100EE0005608F2005708F3005808F4005308831618
:100EF000A100831252088316A0008312AF20033092
:100F0000D0006030D1000130D2002815E32F510805
:100F1000C03C031DB22F0230B4005008023C03183D
:100F2000AA2F3808B80A8316A00083123408B40A1E
:100F3000503E840000088316A200F800903020077D
:100F4000840078088317800083131F308312B8054C
:100F5000D0038D2F0330D0006030D1000230D2009A
:100F60002815E32F5108E03C031DE32F3B08B40094
:100F70003A08B5000712B5080319D42F0230340718
:100F8000503E840000083505003A0319C92F871622
:100F9000CA2F8712A81FCF2F87158711D12F87112E
:100FA00087150310B50CBB2F8030B5003408B4038F
:100FB000003A031DBB2F07160330D0006030D1006C
:0C0FC0000330D20028158A150A12612A9D
:10100000051E0428281C002828182A2800308316CA
:101010008800831250082F02031822282F08AF0AD5
:10102000503E84000008FD0088000714051A1A28A5
:10103000281C16280710051E1F28281C1B2883168D
:1010400009288312FF30831688008312AF0128110C
:10105000091009148A150A12652A051E3128281C50
:101060002D28281865280830D0002030D100D30161
:101070001830D200D4017C08D500D601AF01003071
:1010800083168800831250082F0203185D282F084A
:10109000AF0A503E840000088316A1008312880026
:1010A0000714051A5528281C51280710051E5A2810
:1010B000281C5628831642288312FF308316880086
:1010C0008312AF01281109100914003484011F3064
:1010D000830583161F149F141F159F111F149F143F
:1010E0001F159F111030850000308600D03087001A
:1010F000FF30880002308900811318308312850088
:10110000D03087000730890085120715D33087005B
:10111000D030870089188F28091109158A28AA015B
:10112000A8102811A8112810A812AD01B001B10112
:10113000AC01B801B901E230B6000B30B20010309A
:1011400003178D0083168C130C1483120C080313E1
:10115000C800113003178D0083168C130C148312F2
:101160000C080313C900123003178D0083168C136B
:101170000C1483120C080313CA00133003178D00DC
:1011800083168C130C1483120C080313CB004B082A
:10119000033C031947290330CB00F930CA00403023
:1011A000C900AB30C800103003178D000313480886
:1011B00003178C0083168C130C15831203130B0872
:1011C000F7008B138316031755308D00AA308D005E
:1011D0008C148C18E9280C117708831203138B04E4
:1011E000113003178D000313490803178C00831671
:1011F0008C130C15831203130B08F7008B13831643
:10120000031755308D00AA308D008C148C180629D8
:101210000C117708831203138B04123003178D000F
:1012200003134A0803178C0083168C130C158312C2
:1012300003130B08F7008B138316031755308D002B
:10124000AA308D008C148C1823290C117708831276
:1012500003138B04133003178D0003134B0803177C
:101260008C0083168C130C15831203130B08F700E4
:101270008B138316031755308D00AA308D008C1404
:101280008C1840290C117708831203138B04463005
:10129000A9000E30AB0081010730F700F71D582977
:1012A00007308101813084000008C0390F38800088
:1012B0006400813084000008C039770480008B16F8
:1012C000C0308B042812051A28166030AE008A112F
:1012D0008C208A158A119D208A150930F000033070
:1012E0008316A100A0018A118312AF208A1506304F
:1012F000F00003308316A1000130A0008A11831290
:10130000AF208A15FF30F300F200F100F000033047
:101310008316A1000230A0008A118312AF208A1523
:101320004030F300F201F101F00103308316A10017
:10133000A0008A118312AF208A15F301F201F10196
:10134000F00103308316A1000430A0008A1183123B
:10135000AF208A15F00103308316A1000530A000EC
:101360008A118312AF208A150130F00003308316F2
:10137000A1000630A0008A118312AF208A15083020
:10138000F00003308316A1000730A0008A118312F9
:10139000AF208A15F00103308316A1000830A000A9
:1013A0008A118312AF208A150330F0008316A10042
:1013B0000930A0008A118312AF208A15F001033092
:1013C0008316A1000A30A0008A118312AF208A156B
:1013D000F00103308316A1000B30A0008A118312A4
:1013E000AF208A15F00103308316A1000C30A00055
:1013F0008A118312AF208A15FF30F000F100073008
:10140000F200F301F401F6011130F5007608003C1A
:10141000031C172A76088316A1007508A0008A11FC
:101420008312AF208A15F50A0319F60A062AF0017D
:1014300003308316A1000D30A0008A118312AF2063
:101440008A150930F00003308316A100A0018A112B
:101450008312AF208A150830F00003308316A100F4
:10146000A0018A118312AF208A15CF01FE30CE0071
:101470005030CD002A30CC008A1107218A15051A78
:10148000A52A8A11332B8A158A11752B8A1589187A
:101490005D2A09112A08AA0A503E84000808800023
:1014A00009152A08203C031CAA0350082A02031C21
:1014B0005C2AAA01A8145D2A472AA81C622A8A115C
:1014C000C02B8A15281D662A0028A52AA81DA52A32
:1014D000891CA52A2818A52AAA08031DA52A0910CF
:1014E0000914B1080319932AB00B8F2AA81E832A66
:1014F0008A11F1208A150230FC002D200130FC00F9
:101500002D20A8118E2A3108B0000230FC002D20B9
:101510008A11F1208A158A11F3218A15922A8A11DB
:10152000F3218A15962A8A11F3218A15053083162C
:10153000A0008A118312AD238A152D08AD0AFC0084
:10154000FC18A42A0711A52A0715281CC42A8A11E9
:101550009D208A151C30A9002818BF2A64308316E4
:10156000A0008A118312AD238A15071164308316F7
:10157000A0008A118312AD238A150715AC2A4630C4
:10158000A9002810FC012D20A819D72A2D08AD0A82
:10159000003A031DD12A07113D30F700F70BCE2A80
:1015A000000007154630A9000B30B200D92A0C30D4
:0615B000B2003F2A6300B7
:0602000000006400000094
:02400E003A3F37
:00000001FF
